:0200000480007A
:100000006F008004732F2034930F80006308FF0378
:10001000930F90006304FF03930FB0006300FF038E
:10002000130F000063040F0067000F00732F2034CC
:1000300063540F006F00400093E19153171F0000BD
:1000400023223FFC6FF09FFF93000000130100008C
:10005000930100001302000093020000130300004C
:100060009303000013040000930400001305000034
:10007000930500001306000093060000130700001C
:100080009307000013080000930800001309000004
:1000900093090000130A0000930A0000130B0000EC
:1000A000930B0000130C0000930C0000130D0000D4
:1000B000930D0000130E0000930E0000130F0000BC
:1000C000930F0000732540F16310050097020000B4
:1000D000938202017390523073500018970200000F
:1000E00093824202739052309B021000939252030B
:1000F0009382F2FF7390023B9302F0017390023AF5
:100100007350403097020000938242017390523046
:10011000735020307350303093010000970200007C
:10012000938282EE73905230130510001315F5017F
:10013000635C05000F00F00F930110009308D005D9
:10014000130500007300000093020000638A0200A0
:1001500073905210B7B200009B82921073902230BD
:100160007350003097020000938242017390123462
:10017000732540F17300203097200000938080E8C1
:1001800003C700009303F00F93012000631C772244
:1001900097200000938000E703C71000930300003E
:1001A000930130006310772297200000938080E550
:1001B00003C720009303000F9301400063147720CE
:1001C00097200000938000E403C730009303F00001
:1001D000930150006318771E972000009380B0E2CF
:1001E00003C7D0FF9303F00F93016000631C771CDB
:1001F00097200000938030E103C7E0FF93030000E5
:10020000930170006310771C972000009380B0DF8B
:1002100003C7F0FF9303000F930180006314771A64
:1002200097200000938030DE03C700009303F000A6
:10023000930190006318771897200000938080DC6A
:10024000938000FE83C200029303F00F9301A0008D
:10025000639A7216972000009380C0DA9380A0FF03
:1002600083C27000930300009301B000639C72147A
:100270009301C0001302000097200000938090D8E3
:1002800003C71000130307009303000F631C7312CE
:100290001302120093022000E31052FE9301D000DB
:1002A00013020000972000009380E0D503C71000E0
:1002B00013000000130307009303F000631473108E
:1002C0001302120093022000E31E52FC9301E0008F
:1002D00013020000972000009380C0D203C71000D3
:1002E0001300000013000000130307009303000035
:1002F000631A730C1302120093022000E31C52FCD9
:100300009301F0001302000097200000938090CF2B
:1003100003C710009303000F6316770A130212003D
:1003200093022000E31252FE930100011302000029
:1003300097200000938020CD1300000003C7100019
:100340009303F00063107708130212009302200059
:10035000E31052FE930110011302000097200000E9
:10036000938040CA130000001300000003C7100070
:100370009303000063187704130212009302200015
:10038000E31E52FC972200009382C2C703C1020001
:1003900013012000930320009301200163147102D4
:1003A00097220000938202C603C1020013000000DE
:1003B00013012000930320009301300163147100A6
:1003C000631030020F00F00F638001009391110061
:1003D00093E111009308D00513850100730000001C
:1003E0000F00F00F930110009308D00513050000D3
:0C03F00073000000731000C0000000004B
:1010000000000000000000000000000000000000E0
:1010100000000000000000000000000000000000D0
:1010200000000000000000000000000000000000C0
:1010300000000000000000000000000000000000B0
:081040000000000000000000A8
:10200000FF00F00F000000000000000000000000D2
:040000058000000077
:00000001FF
